:020000040000FA
:040000003EEF02F0DD
:08000800E8CF05F0D8CF06F0A7
:10001000E0CF07F00001E9CF0DF0EACF08F0E1CF23
:1000200009F0E2CF0AF0D9CF0BF0DACF0CF0F3CF22
:1000300014F0F4CF15F0FACF16F000C00FF001C0A5
:1000400010F002C011F003C012F004C013F09DAA1A
:100050002DEF00F09EBA9CEF00F00FC000F010C032
:1000600001F011C002F012C003F013C004F00DC083
:10007000E9FF08C0EAFF09C0E1FF0AC0E2FF0BC0C8
:10008000D9FF0CC0DAFF14C0F3FF15C0F4FF16C08F
:10009000FAFF05C0E8FF07C0E0FF06C0D8FF100068
:1000A000F2CF0EF0F29EF76ABA0FF66E000EF7224C
:1000B0000900F5500EBEF28E1200496E6974696136
:1000C0006C697A696E6720506F727420420A0D0065
:1000D000F2CF0EF0F29EF76AEA0FF66E000EF722EC
:1000E0000900F5500EBEF28E1200436F6E6669670E
:1000F0007572696E672052462D3234470A0D000032
:10010000F2CF0EF0F29EF76A1A0FF66E010EF7228A
:100110000900F5500EBEF28E12004F4B210A0D0061
:100120009EAAFED7ABCF18F0AECF01F018A202D036
:10013000AB98AB880000000C9D9AF29CF29EF2BE38
:10014000FDD7EEDF01C026F101012651120A0001A0
:1001500001E02DD0E5DF0150340802E0000E01D0AF
:10016000010E0101286F0001DBDF0150560802E09B
:10017000000E01D0010E010128152A6F0001D0DF09
:100180000150780802E0000E01D0010E01012A158D
:100190002C6F0001C5DF0150900802E0000E01D075
:1001A000010E01012C15D8A4FF000DD000011B0E7B
:1001B00001011B25E96EEA6AD8B0EA2A26C1EFFFE1
:1001C0001B2B1E2B00D09D8AC00EF2129E9A00019E
:1001D0002DEF00F0010EEA6E1F0EE96EEF500FE0FA
:1001E000030E016E006A002EFED7012EFBD73C0ED7
:1001F000006E002EFED700000000EF2EF1D7000C9D
:10020000070E0101236F226B225107081DE3939A09
:100210008A9A23512307246F21C100F02451016ED3
:1002200004E0D8900032012EFCD700A003D09398B0
:100230008A8802D093988A9800000000939A8A8A4C
:1002400000000000222BE0D70001000C93968A9654
:10025000939E8A9E939A8A9A93988A98030E010194
:100260001F6F0001B7DF939E8A8E080E006E002E6E
:10027000FED7100E0101216F0001C2DF100E010137
:10028000216F0001BDDF0101216B0001B9DF010118
:10029000216B0001B5DF0101216B0001B1DF420ECE
:1002A0000101216F0001ACDF420E0101216F00014D
:1002B000A7DF0101216B0001A3DF0101216B000118
:1002C0009FDF0101216B00019BDF420E0101216FC5
:1002D000000196DF420E0101216F000191DF430E04
:1002E0000101216F00018CDF6F0E0101216F000100
:1002F00087DF810E0101216F000182DF93889396D1
:100300008A96939E8A9E939A8A9AB3EF02F0939666
:100310008A96939E8A8E080E006E002EFED79398C2
:100320008A88939A8A8A00000000939A8A9A000029
:100330000000939E8A9E9388939A8A9A93968A86BF
:10034000000C0101236B070E246F226B225107085A
:100350002BE3939A8A9A00000000939A8A8A0000FD
:100360000000938881A80FD024512407256F010E27
:10037000006E2551016E04E0D8900036012EFCD7A6
:10038000005023130FD024512407256F010E006E57
:100390002551016E04E0D8900036012EFCD70050A4
:1003A000FF0A2317222BD2D723C101F00001EAEF65
:1003B00001F001011F6B1F51010815E3036A1F5172
:1003C000190F016E000E032201C020F103C021F1BC
:1003D0000001B7D721C1EAFF20C1E9FF01C0EFFF4B
:1003E00001011F2BE8D7939A8A9A93968A86000177
:1003F000CCEF02F093968A96939E8A8E080E006E3A
:10040000002EFED793988A98939A8A8A000000005B
:10041000939A8A9A00000000939E8A9E939A8A9AE1
:10042000E0EF02F093968A86080E006E002EFED74B
:10043000420E0101216F0001E3DE420E0101216F36
:100440000001DEDE01011F6B1F51010810E3036A8A
:100450001F51190FE96E000E0320EA6EEFCF20F155
:1004600020C121F10001CCDE01011F2BEDD79396B5
:100470008A96939A8A9A0001E6EF02F0F86AD09E73
:100480000D8EEA6AE96AB8862A0EAF6E000EB06E6B
:10049000260EAC6E900EAB6EC150C00B0F09C16E34
:1004A000070EB46E186A01011B6B1C6B1D6B1E6B73
:1004B000C150C00B0F09C16EC290880ED56ECD6AB7
:1004C000000ECA6E7F0ECB6EB150480BB16EB70EE8
:1004D000B1169484BD6ABD6AB1169482BA6ABA6ACA
:1004E0009D8AC00EF2121F6B1F510001D9DD010160
:1004F0001F2B006E00509EA8FED7AD6E130E1F5D21
:10050000F3E1030E206F2E0E9EA8FED7AD6E202FB6
:10051000FAD70A0E9EA8FED7AD6E0D0E9EA8FED786
:10052000AD6EF18EF2961F6B1F510001D1DD0101FE
:100530001F2B006E00509EA8FED7AD6E120E1F5DE1
:10054000F3E1030E206F2E0E9EA8FED7AD6E202F76
:10055000FAD70A0E9EA8FED7AD6E0D0E9EA8FED746
:10056000AD6E000173D6D3DE410E196E420E1A6EC7
:1005700001011F6B1F510001C3DD01011F2B006E24
:1005800000509EA8FED7AD6E050E1F5DF3E1938C63
:1005900081AC07D000010DD719509EA8FED7AD6ED3
:1005A00001011C511B5D1EE01B0E1C25E96EEA6A51
:1005B000D8B0EA2AEFCF19F01C2B1E0700011AD77A
:1005C000010E01011F6F000105DE2CD7010E010194
:1005D0001F6F0001FFDD9BDE010E01011F6F000197
:0805E000F9DD0101D4D703008D
:00000001FF
